:02000000632873
:0800080005280B181B288B18BA
:100010000A2808000B1206088B1094210608AB0072
:100020002B1814280330A5005B20CC3025083D0890
:100030000B168B1732288B1106080B10942106081B
:10004000AB002B08AB1B26280130A5002B082B1B6F
:100050002B280230A5005B209E212508B4203D08F6
:100060008B158B1701303C0603191E210130250624
:10007000031D4228000001303D06031DE628003024
:10008000BD005A2802302506031D4E28000002300C
:100090003D06031D01290030BD005A280330250606
:1000A000031D5A28000003303D06031D0B290030B4
:1000B000BD005A28A328942106090B108B15C139BD
:1000C000031908005B2800000130A600A700A80063
:1000D000B400B500B600B700B800B900BA01BB0162
:1000E0000030BC00BD00413084005A30C1000130F6
:1000F000C2001630C3002D30C4001630C5001630C3
:10010000C6001630C700850107309F008316D73020
:1001100086008113011383128B1106080B108B15B7
:100120008B100B1683129817181683161930990026
:100130001815981683128B171A081A081A08003017
:10014000AC001F30AE0000000000000086169E21AB
:1001500086129E219E219E219E21A3281430AD004F
:100160001430AF002621080099000C1EB5280800A5
:10017000333099000C1EBA280800413099000C1E3B
:10018000BF289E210800423099000C1EC5289E21E0
:100190000800433099000C1ECB289E2108004430F3
:1001A00099000C1ED1289E21080085009E219E21C9
:1001B000003085009E21080082070034013402349B
:1001C0000434083410342034403480340130BD000D
:1001D000AA3023212608AB2123212608AB21232185
:1001E0002608AB2123212608AB2123212608AB2199
:1001F00023212608AB2119212608AB211E219E218F
:10020000E62800000230BD0019210330AB211E2179
:100210000330AB21012900000330BD001921033058
:10022000AB211E219E210030BD00A3280B302621CA
:1002300008000130BC001430262108000030BC004A
:100240001430262108001030262108000000AC00E0
:100250000330AA002C08B1000730B0004521B10CD2
:1002600003184C21031C5121B00B2F290130B2007F
:100270000530B000B20C03184C21031C5121B00B07
:100280003A299821AA0B2A29003441085921420809
:100290005921430874210034440859214508742128
:1002A0000034460859214708742100341730592179
:1002B0000034A400861600000000000000000000CA
:1002C0000000000000000000000000008612000096
:1002D000000000000000000000000000000000001E
:1002E0000000A40B5A290034A4008612000000006C
:1002F00000000000000000000000000000000000FE
:100300000000861200000000000000000000000055
:100310000000000000000000A40B75290034003428
:1003200001309F2905309F290A309F2914309F29C9
:100330002D309F2932309F2964309F29FA30A00048
:10034000C730A1000130A200A10BA729A20BA4294C
:10035000A00BA0290034A300FA30A000C730A100F0
:10036000BB30A200A10BB529A20BB229A00BAE296C
:10037000A30BAC290034A3007D30A000C730A1003E
:10038000BB30A200A10BC529A20BC229A00BBE291C
:06039000A30BBC290034A0
:02400E00B003FD
:00000001FF
